:020000040000FA
:100000008316031386012030A00010309A009B0154
:100010002F209A0A9B0AA00B08282030A0009B01E1
:100020003D208312031386002B20831603139B0AA3
:10003000A00B102863001930A200A100A10B1E28FC
:10004000A20B1D280800FA30A200A100A10B26284F
:10005000A20B252808002320232023200800831634
:1000600003131C158B1355309D00AA309D009C1462
:100070009C1838281C118B170800831603131C14B6
:040080001A08080052
:02400E00293F48
:00000001FF
